:10000000C2C0DCC0DBC0DAC0D9C0D8C0D7C0D6C03F
:10001000D5C034C1D3C0D2C0D1C0D0C0CFC0CEC0F3
:10002000CDC0CCC0CBC02300E8030000E1024B00F0
:1000300053564E203733310076302E316200496EF0
:10004000666F726D6174696F6E656E002533640052
:100050002525004D61782E20447265687A61686CB0
:100060000025346400253464002D005265676C65FA
:1000700072206265776567656E00253464002534FB
:1000800064002D004675E2706564616C20626577DE
:100090006567656E00447265687265676C657200BD
:1000A0004675E2706564616C20200045696E676189
:1000B0006265676572E1743A00286D6F6D656E74F4
:1000C000616E202533642525293F004D61782E205F
:1000D000447265687A61686C006B616C6962726910
:1000E0006572656E3F00447265687265676C657223
:1000F000006B616C696272696572656E3F0046757E
:10010000E2706564616C002533640025632025334B
:1001100064002533640025336400537461727400F5
:1001200053544F502000DF4300DF430025250025B6
:10013000252F005E5E5E5E5E5E5E5E5E5E0046F584
:1001400072204A756C616961005E5E5E5E5E5E5E35
:100150005E5E5E5E5E5E004A6F65277320456C736F
:100160007069726100FF7A63564D47413D393532FF
:100170002F2D2A28262422201E1D1B1A181615147E
:1001800012110F0E0D0011241FBECFE5D4E0DEBF0B
:10019000CDBF10E0A0E6B0E0EEE0F9E102C00590CE
:1001A0000D92AC37B107D9F710E0ACE7B0E001C071
:1001B0001D92AF39B107E1F702D0A7CB21CF909ABA
:1001C00088989198899A92988A9A93988B9AC098CD
:1001D000B89A949A8C98959A8D98969A8E98979AA0
:1001E0008F98C198B99AC29ABA98A898A098A998D5
:1001F000A198AA98A298AB98A398AC9AA498AD9A03
:10020000A598F7D39CD74FD814D084D0E7D024D862
:100210002DD37894A5D1FECF97B1907F97B997B1A0
:10022000982B97B9369A3699FECF24B135B1C901CA
:10023000089580EC87B987E886B90895282F30E0C3
:10024000D901A458BF4F8C916817B9F0F901E25851
:10025000FF4F662361F090819F5F9083963069F431
:1002600081E08C9320583F4FF9018083089580816D
:1002700081508083882309F41C9208951F920F9265
:100280000FB60F9211242F933F934F935F936F9369
:100290007F938F939F93AF93BF93CF93DF93EF930E
:1002A000FF9363B370E094E0769567959A95E1F7D4
:1002B000C1E0D0E06C277D27617080E0BFDF63B3D1
:1002C00070E085E0769567958A95E1F76C277D2744
:1002D000617081E0B3DFFF91EF91DF91CF91BF912A
:1002E000AF919F918F917F916F915F914F913F91CE
:1002F0002F910F900FBE0F901F90189510928000B5
:10030000109281000895E0E8F0E0E80FF11D80818F
:100310001082089584E083BF89B7816089BF089502
:1003200008DA08950F931F93CF93DF938C01C0E0F9
:10033000D0E0CE01FED9F801EC0FFD1F808321969D
:10034000CA30D105B1F7DF91CF911F910F91089578
:10035000F8D90895EF92FF920F931F93CF93DF93F5
:100360008C01C0E0D0E0F801EC0FFD1FCE016081F0
:10037000E8D92196CA30D105B1F7F8019801265F76
:100380003F4FCFEFDFEF8191C8278C2F82958C27CD
:10039000082E869586958025082E8695802587705F
:1003A0000C2ECD2F869507948795D02DC8270694BF
:1003B0008795D025C827E217F30729F78AE090E050
:1003C0007E016C2FBED98BE090E06F2DBAD9DF9102
:1003D000CF911F910F91FF90EF900895FF920F938F
:1003E0001F93DF93CF93CDB7DEB72A970FB6F8945C
:1003F000DEBF0FBECDBF8E010F5F1F4FC80192DF62
:10040000F8019E01255F3F4F0FEF1FEF81910827F5
:10041000802F82958027082E869586958025082E28
:10042000869580258770002E012F869507948795E5
:10043000102D08270694879510250827E217F30743
:1004400029F78AE090E075D9F82E8BE090E071D919
:10045000382F20E08F2D90E0822B932B081719075F
:1004600059F08E010F5F1F4FC80166E270E04AE04D
:1004700050E079D7C8016EDF2A960FB6F894DEBF38
:100480000FBECDBFCF91DF911F910F91FF900895C7
:100490008091830008958091840008958091950053
:1004A0000895809185000895809186000895809137
:1004B000870090E0089580918800909189000895C8
:1004C00080918A0090918B00089580919600089504
:1004D000CF93DF93EC0180E090E02881398140E008
:1004E00050E0ECD62A813B8140E050E01AD7C901A8
:1004F000DF91CF910895EF92FF920F931F93CF93C7
:10050000DF93EC01862F623049F400919100109145
:100510009200E0909300F090940008C000918D004C
:1005200010918E00E0908F00F090900075DE9701A2
:10053000201B310B3B832A838017910710F4C801DD
:1005400004C0E816F90608F4C701801B910B9983D3
:100550008883DF91CF911F910F91FF90EF900895C5
:100560000F931F93DF93CF9300D000D0CDB7DEB7AA
:1005700000918200002309F057C080E0C4DE882388
:1005800069F080918300882321F481E080938300C7
:1005900005C01092830080E090E05BD680E03CDEF6
:1005A00029D68093850081E037DE24D680938600AB
:1005B00080919600882311F062E001C063E08E0113
:1005C0000F5F1F4FC80197DF60919500C80170E071
:1005D0007FDF8093840080918300813091F436D650
:1005E0002091950030E0AC01429FC001439F900DE7
:1005F000529F900D112464E670E07FD6C80168DF39
:1006000028D680918C0082D410928C0081E07BDE11
:10061000882309F422C181E08093820080938C00BA
:1006200080E090E016D619C1013001F580918C0070
:1006300084D210928C0080E066DE882361F08FEF18
:100640009FEF909389008093880010928B00109206
:100650008A0086E006C081E056DE882309F4FDC0EA
:1006600082E08093820000938C00F7C00230D9F4BE
:1006700080918C0033D210928C0080E044DE88237D
:1006800061F08FEF9FEF9093890080938800109224
:100690008B0010928A0087E0DBC081E034DE882383
:1006A00009F4DBC0D4C0033091F480918C00EED308
:1006B00010928C0080E027DE882311F088E0C8C00B
:1006C00081E021DE882309F4C8C084E0C1C0043081
:1006D000F1F480918C009AD310928C0080E013DEAC
:1006E000882371F080919600882321F481E0809323
:1006F000960002C0109296008DE890E02BDEADC00F
:1007000081E001DE882309F4A8C085E0A1C005309E
:1007100069F480918C00A1D110928C0081E0F3DD0E
:10072000882309F49AC01092820094C00630C9F55B
:1007300083E072DD20918800309189008217930751
:1007400020F4909389008093880020918A00309152
:100750008B002817390720F490938B0080938A0030
:1007600080918C00E0D210928C0080E0CCDD882358
:1007700009F473C0809188009091890090938E0055
:1007800080938D0080918A0090918B0090939000CF
:1007900080938F008DE890E0DDDD81E08093820022
:1007A0005AC00730B1F582E037DD209188003091E2
:1007B00089008217930720F4909389008093880022
:1007C00020918A0030918B002817390720F49093EC
:1007D0008B0080938A0080918C0032D210928C0022
:1007E00080E091DD8823C9F1809188009091890093
:1007F000909392008093910080918A0090918B0059
:1008000090939400809393008DE890E0A3DD82E0C4
:100810001FC0083011F58E010F5F1F4FC80162E045
:100820006ADEC80164E670E053DE80938700809141
:100830008C00B2D110928C0080E065DD882369F0D5
:1008400080918700809395008DE890E083DD83E0C0
:100850008093820081E080938C000F900F900F9026
:100860000F90CF91DF911F910F9108951092820008
:10087000109283001092840081E080938C008DE8B8
:1008800090E050DD089526E63EE004C0F90131977E
:10089000F1F701970097D1F7089593988C9A8D9A64
:1008A0008E9A8F9A662311F0929A01C0929840FF17
:1008B00002C0949A01C0949841FF02C0959A01C069
:1008C000959842FF02C0969A01C0969843FF02C0D5
:1008D000979A01C09798C09A81E090E0D4DFC098C1
:1008E00081E090E0D0DF08958C988D988E988F9855
:1008F0009498959896989798939A9298C09A81E030
:1009000090E0C1DF90B340B320B380B3C098991F8B
:100910009927991F990F990F990F50E040745070C3
:10092000E6E055954795EA95E1F7440F551F440FCA
:10093000551F942B482F50E04071507064E055953E
:1009400047956A95E1F7942B30E02072307045E0CE
:10095000359527954A95E1F7220F331F892F822B72
:1009600008951F9380919700882341F0BDDF182FD1
:100970001295107FB9DF812B87FDF8CF1F91089565
:10098000FF920F931F93182FF62E042FEADF402FAC
:1009900042954F70812F6F2D80DF812FE2DF812FF5
:1009A0006F2D402F7ADF1F910F91FF900895482FF0
:1009B0008091980061E0E4DF0895F9DF81E090E044
:1009C0000895482F623028F410929800613031F079
:1009D00006C081E080939800633009F4405C809108
:1009E0009800406860E0CCDF089560E041E0C8DF37
:1009F000089580E190E047DF1092970080E060E08A
:100A000043E04BDF85E090E03EDF80E060E043E0E4
:100A100044DF81E090E037DF80E060E043E03DDFED
:100A200085E090E030DF80E060E042E036DF81E0AA
:100A30008093970080E060E048E2A2DF80E060E021
:100A40004CE09EDF80E0D1DF80E060E042E098DFB4
:100A500080E060E046E094DF0895CF93DF93882341
:100A6000D1F180E0C2DF81E060E0ABDF00D000D0F8
:100A7000C0E6D0E0EDB7FEB7D283C1838EE390E04D
:100A80009483838379D40F900F900F900F9081E01F
:100A900061E097DF00D000D0EDB7FEB7D283C1830D
:100AA00088E390E09483838367D40F900F900F9036
:100AB0000F9087E061E085DF00D000D0EDB7FEB792
:100AC000D283C18380E390E09483838355D40F90D5
:100AD0000F900F900F90DF91CF910895CF93DF93F8
:100AE000882341F180E081DF81E060E06ADF00D0AF
:100AF00000D0C0E6D0E0EDB7FEB7D283C18386EE6A
:100B000090E09483838338D40F900F900F900F90D0
:100B100081E061E056DF00D000D0EDB7FEB7D283B0
:100B2000C18389ED90E09483838326D40F900F9046
:100B30000F900F90DF91CF910895CF93DF9388238B
:100B400041F180E052DF81E060E03BDF00D000D087
:100B5000C0E6D0E0EDB7FEB7D283C1838EEF90E060
:100B60009483838309D40F900F900F900F9081E0AE
:100B700061E027DF00D000D0EDB7FEB7D283C1839C
:100B800081EF90E094838383F7D30F900F900F90C1
:100B90000F90DF91CF910895CF93DF93882361F178
:100BA00080E023DF81E060E00CDF00D000D0C0E611
:100BB000D0E0ADB7BEB71296DC93CE93119783E524
:100BC00090E014969C938E931397D6D30F900F902A
:100BD0000F900F9087E061E0F4DE00D000D0EDB719
:100BE000FEB7D283C18380E590E094838383C4D32E
:100BF0000F900F900F900F9084E061E0E2DE57DCE1
:100C000000D000D000D0EDB7FEB7319620E630E03E
:100C1000ADB7BEB712963C932E9311972CE430E0FB
:100C20003383228395838483A7D3EDB7FEB73696AB
:100C30000FB6F894FEBF0FBEEDBFDF91CF910895C0
:100C4000CF93DF93882361F180E0CFDE80E060E026
:100C5000B8DE00D000D0C0E6D0E0ADB7BEB7129687
:100C6000DC93CE9311978BE690E014969C938E9331
:100C7000139782D30F900F900F900F9087E061E051
:100C8000A0DE00D000D0EDB7FEB7D283C18389E6E5
:100C900090E09483838370D30F900F900F900F9008
:100CA00082E061E08EDE07DC00D000D000D0EDB73E
:100CB000FEB73196C0E6D0E0ADB7BEB71296DC9372
:100CC000CE93119725E630E0338322839583848386
:100CD00053D3EDB7FEB736960FB6F894FEBF0FBEEE
:100CE000EDBF89E061E06DDEEBDB00D000D000D02D
:100CF000EDB7FEB73196ADB7BEB71296DC93CE9383
:100D0000119721E630E0338322839583848334D3A3
:100D1000EDB7FEB736960FB6F894FEBF0FBEEDBF27
:100D2000DF91CF910895CF93DF93882361F180E025
:100D30005CDE80E060E045DE00D000D0C0E6D0E0C0
:100D4000ADB7BEB71296DC93CE93119784E890E0CE
:100D500014969C938E9313970FD30F900F900F9030
:100D60000F9087E061E02DDE00D000D0EDB7FEB738
:100D7000D283C18382E890E094838383FDD20F9075
:100D80000F900F900F9082E061E01BDE94DB00D0AB
:100D900000D000D0EDB7FEB73196C0E6D0E0ADB7D9
:100DA000BEB71296DC93CE9311972EE730E03383D3
:100DB000228395838483E0D2EDB7FEB736960FB6D3
:100DC000F894FEBF0FBEEDBF89E061E0FADD78DB8D
:100DD00000D000D000D0EDB7FEB73196ADB7BEB7AA
:100DE0001296DC93CE9311972AE730E03383228367
:100DF00095838483C1D2EDB7FEB736960FB6F894CB
:100E0000FEBF0FBEEDBFDF91CF910895CF93DF936B
:100E10008823B1F080E0E9DD81E060E0D2DD00D040
:100E200000D080E690E0EDB7FEB7928381838BEA35
:100E300090E094838383A0D20F900F900F900F9037
:100E400044DBC0E6D0E0882361F483E061E0B9DDF3
:100E500000D000D0EDB7FEB7D283C18380EA90E026
:100E60000BC083E061E0ADDD00D000D0EDB7FEB790
:100E7000D283C18385E990E0948383837DD20F90F0
:100E80000F900F900F90DF91CF910895CF93DF9344
:100E90008823C9F180E0A9DD81E060E092DD00D027
:100EA00000D0C0E6D0E0ADB7BEB71296DC93CE93CB
:100EB00011978BEC90E014969C938E9313975CD2D1
:100EC0000F900F900F900F9081E061E07ADDE6DAED
:100ED00000D000D000D0EDB7FEB73196ADB7BEB7A9
:100EE0001296DC93CE93119729EB30E03383228363
:100EF0008483158241D2EDB7FEB736960FB6F894CB
:100F0000FEBF0FBEEDBFDF91CF9108950F931F93EA
:100F1000CF93DF93882309F454C080E066DD83E03B
:100F200061E04FDD00D000D0C0E6D0E0ADB7BEB785
:100F30001296DC93CE9311978FE291E014969C93D6
:100F40008E93139719D20F900F900F900F9088E007
:100F500061E037DD00D000D0EDB7FEB7D283C183AA
:100F60008CE291E09483838307D20F900F900F90CF
:100F70000F908EE060E025DD00D000D0ADB7BEB7A9
:100F80001296DC93CE93119789E291E014969C938C
:100F90008E931397F1D10F900F900F900F908EE0DA
:100FA00061E00FDD00D000D0EDB7FEB7D283C18382
:100FB00086E291E094838383DFD10F900F900F90AE
:100FC0000F9066DAC0E6D0E0882391F482E060E01A
:100FD000F8DC00D000D0ADB7BEB71296DC93CE934C
:100FE000119780E291E014969C938E9313970DC015
:100FF00082E060E0E6DC00D000D0EDB7FEB7D2833F
:10100000C1838AE191E094838383B6D10F900F90DE
:101010000F900F9080E061E0D4DC3DDA00D000D08A
:1010200000D0EDB7FEB73196C0E6D0E0ADB7BEB7A1
:101030001296DC93CE93119726E131E0338322831D
:101040008483158299D1EDB7FEB736960FB6F89422
:10105000FEBF0FBEEDBF85E061E0B3DC1FDA00D05C
:1010600000D000D0EDB7FEB73196ADB7BEB712963F
:10107000DC93CE93119722E131E033832283848382
:1010800015827AD1EDB7FEB736960FB6F894FEBF4B
:101090000FBEEDBF89E060E094DC17DA882319F019
:1010A00004E410E002C006E410E0FBD92DB73EB71F
:1010B000285030400FB6F8943EBF0FBE2DBFEDB79D
:1010C000FEB73196C0E6D0E0ADB7BEB71296DC935E
:1010D000CE9311972BE031E0338322831583048371
:1010E0008683178249D1EDB7FEB738960FB6F894CC
:1010F000FEBF0FBEEDBF8BE061E063DCD5D900D051
:1011000000D000D0EDB7FEB73196ADB7BEB712969E
:10111000DC93CE93119727E031E0338322838483DD
:1011200015822AD1EDB7FEB736960FB6F894FEBFFA
:101130000FBEEDBFDF91CF911F910F910895CF9317
:10114000DF9380E052DC81E060E03BDC00D000D047
:10115000C0E6D0E0EDB7FEB7D283C18387E591E06A
:101160009483838309D10F900F900F900F9081E0AB
:1011700061E027DC00D000D0EDB7FEB7D283C18399
:1011800089E491E094838383F7D00F900F900F90C0
:101190000F908CED95E077DB80E027DC83E060E06A
:1011A00010DC00D000D0EDB7FEB7D283C1838EE350
:1011B00091E094838383E0D00F900F900F900F9075
:1011C00083E061E0FEDB00D000D0EDB7FEB7D28354
:1011D000C18383E391E094838383CED00F900F90FB
:1011E0000F900F908CED95E04EDB80E0FEDBDF9101
:1011F000CF910895FC0195E0F695E7959A95E1F772
:101200005E2F2E2F30E0EF31E0F4482F4F712B5935
:101210003E4FF9012491E52FEF5FF0E0EB59FE4FCF
:10122000E491E49FF00111249FE1941B299F900118
:101230001124CF01820F931F6FE170E05ED0862FE3
:1012400008952B593E4FF901849108958CEE91E059
:1012500008959BBD8ABD08951BBC1ABC8CEE91E01D
:1012600097BD86BD80E88FBD81E18EBD08955D9BF1
:10127000FECF8CB981E090E008955D9BFECF8CB9E4
:1012800008955F9BFECF8CB108955F9903C00197CD
:10129000E1F705C0009719F02CB130E002C02FEF44
:1012A0003FEFC901089587E089B988E18AB98EE6E0
:1012B00090E090939C0080939B000895629FD001E2
:1012C000739FF001829FE00DF11D649FE00DF11D01
:1012D000929FF00D839FF00D749FF00D659FF00DB0
:1012E0009927729FB00DE11DF91F639FB00DE11D9D
:1012F000F91FBD01CF0111240895AA1BBB1B51E1A9
:1013000007C0AA1FBB1FA617B70710F0A61BB70B75
:10131000881F991F5A95A9F780959095BC01CD011A
:101320000895A1E21A2EAA1BBB1BFD010DC0AA1F26
:10133000BB1FEE1FFF1FA217B307E407F50720F03E
:10134000A21BB30BE40BF50B661F771F881F991FB9
:101350001A9469F760957095809590959B01AC0102
:10136000BD01CF010895FB01DC0102C005900D9283
:1013700041505040D8F70895A0E0B0E0E1ECF9E02A
:101380009BC20F8118859E01255F3F4FF801838125
:1013900088608383C80169857A85A90107D0F8012F
:1013A0002381277F23832096E4E0A2C2ACE0B0E053
:1013B000EBEDF9E074C26C012B018A01FC0117828C
:1013C0001682838181FD03C02FEF3FEFAEC14E0136
:1013D0000894811C911C6FE3362EF6019381F20173
:1013E00093FD859193FF81912F01882309F49AC180
:1013F000853239F493FD859193FF81912F018532D8
:1014000021F490E0B601C0D1E8CFEE24FF2420E023
:10141000203298F4803259F0833269F08B3231F007
:101420008D3239F0803349F421602CC02260246071
:1014300029C0286027C0206125C027FD2CC0382F77
:1014400030533A3098F426FF08C08E2D880FE82ECE
:10145000EE0CEE0CE80EE30E15C08F2D880FF82E63
:10146000FF0CFF0CF80EF30E20620CC08E3221F43C
:1014700026FD58C1206406C08C3611F4206802C0D5
:10148000883649F4F20193FD859193FF81912F01F4
:10149000882309F0BDCF982F9554933018F09052BF
:1014A000933020F40C5F1F4F39820DC0833519F142
:1014B000833621F0833709F054C00AC0F8018081D7
:1014C00089830E5F1F4F540151E0652E712C11C0AE
:1014D000F801A080B18026FD03C06FEF7FEF02C04E
:1014E0006E2D70E00E5F1F4FC5012C8742D13C016D
:1014F0002C852F7712C0F801A080B18026FD03C093
:101500006FEF7FEF02C06E2D70E00E5F1F4FC501C1
:101510002C8724D13C012C85206823FF08C01DC0E6
:1015200080E290E0B6012C872FD1FA942C858F2D84
:1015300090E068167906A0F310C0F50127FD8591AB
:1015400027FF81915F0190E0B6012C871DD12C858A
:10155000F110FA940894610871086114710469F734
:10156000DEC0843611F0893649F527FF08C0F8013E
:1015700060817181828193810C5F1F4F0AC0F801E5
:1015800040815181BA01882777FD8095982F0E5FA1
:101590001F4F4FE6B42EB22297FF09C09095809559
:1015A000709561957F4F8F4F9F4FF0E8BF2AA40140
:1015B0002AE030E015D1782E78183EC0853731F416
:1015C0003FEEB32EB2222AE030E01FC099EFB92ED1
:1015D000B2228835A1F08F3631F0803739F0883764
:1015E00009F0A0C005C028E030E00FC020E1B22A19
:1015F000B4FE02C084E0B82A20E130E006C0B4FEA8
:1016000002C0E6E0BE2A20E132E0B7FE08C0F801E1
:1016100060817181828193810C5F1F4F07C0F80147
:101620006081718180E090E00E5F1F4FA401D8D0EF
:10163000782E7818FFE7BF22B6FE0BC02EEFB2223D
:101640007E1438F4B4FE07C0B2FC05C08FEEB82299
:1016500002C0A72C01C0AE2C8B2DB4FE0DC0FE0124
:10166000E70DF11D9081903319F4E9EEBE2207C019
:10167000A394B2FE04C002C0867809F0A3946B2C38
:10168000B3FC13C0B0FE0EC0AF1410F0E72C0AC0BC
:10169000E72CEF0CEA18AF2C05C080E290E0B60111
:1016A00073D0A394AF14C8F304C0AF1410F4FA18A5
:1016B00001C0FF2464FE0EC080E390E0B60164D058
:1016C00062FE1BC061FC03C088E790E00EC088E5A5
:1016D00090E00BC0862D867881F061FE02C08BE21F
:1016E00001C080E2B7FC8DE290E0B6014DD005C0AC
:1016F00080E390E0B60148D0EA947E14C8F37A946F
:10170000F401E70DF11D808190E0B6013DD0772016
:10171000B1F705C080E290E0B60136D0FA94FF2020
:10172000C9F75BCEF60126813781C9012C96E1E12C
:10173000D2C0E199FECF9FBB8EBBE09A99278DB3B3
:101740000895262FE199FECF9FBB8EBB2DBB0FB610
:10175000F894E29AE19A0FBE01960895FC01059073
:10176000615070400110D8F7809590958E0F9F1FA3
:101770000895FC016150704001900110D8F78095E8
:1017800090958E0F9F1F08950F931F93CF93DF9314
:101790008C01EB018B8181FF1BC082FF0DC02E816C
:1017A0003F818C819D812817390764F4E881F98194
:1017B0000193F983E88306C0E885F985802F0995B0
:1017C000009731F48E819F8101969F838E8302C0A2
:1017D0000FEF1FEFC801DF91CF911F910F91089577
:1017E000FA01AA27283051F1203181F1E8946F9352
:1017F0006E7F6E5F7F4F8F4F9F4FAF4FB1E03ED0F8
:10180000B4E03CD0670F781F891F9A1FA11D680F95
:10181000791F8A1F911DA11D6A0F711D811D911DC8
:10182000A11D20D009F468943F912AE0269F11243D
:101830003019305D3193DEF6CF010895462F4770A1
:10184000405D4193B3E00FD0C9F7F6CF462F4F70FC
:10185000405D4A3318F0495D31FD4052419302D05A
:10186000A9F7EACFB4E0A695979587957795679500
:10187000BA95C9F700976105710508959B01AC0100
:101880000A2E06945795479537952795BA95C9F727
:10189000620F731F841F951FA01D08952F923F9202
:1018A0004F925F926F927F928F929F92AF92BF9270
:1018B000CF92DF92EF92FF920F931F93CF93DF931C
:1018C000CDB7DEB7CA1BDB0B0FB6F894DEBF0FBE79
:1018D000CDBF09942A88398848885F846E847D84C6
:1018E0008C849B84AA84B984C884DF80EE80FD80C8
:1018F0000C811B81AA81B981CE0FD11D0FB6F8943E
:0E190000DEBF0FBECDBFED010895F894FFCFFE
:10190E000000000200000000DD04000000000000E6
:0C191E000002000000003709000000007B
:00000001FF
